:020000040000FA
:100000000C945D000C9485000C9485000C94850084
:100010000C9485000C9485000C9485000C9485004C
:100020000C9485000C9485000C9485000C9485003C
:100030000C9485000C9485000C9485000C9485002C
:100040000C9452070C9485000C9420070C94FA062B
:100050000C9485000C9485000C9485000C9485000C
:100060000C949C070C94850000000008000201001D
:100070000003040700000000000000000000000072
:10008000250028002B0000000000240027002A0083
:10009000040404040404040402020202020203032E
:1000A0000303030301020408102040800102040836
:1000B0001020010204081020BB0811241FBECFEF3E
:1000C000D8E0DEBFCDBF11E0A0E0B1E0EAEBF9E19E
:1000D00002C005900D92A633B107D9F722E0A6E33E
:1000E000B1E001C01D92A53AB207E1F710E0CDE5FD
:1000F000D0E004C02197FE010E94D50CCC35D10779
:10010000C9F70E94FC080C94DB0C0C94000090E0F2
:10011000FC01EC55FF4F249180579F4FFC018491C7
:10012000882399F090E0880F991FFC01EA57FF4F50
:10013000A591B491FC01E458FF4F859194918FB73C
:10014000F894EC91E22BEC938FBF089508950895F5
:10015000AF92BF92CF92DF92EF92FF920F931F93D5
:10016000CF93DF936C017B018B01040F151FEB0113
:100170005E01AE18BF08C017D10759F06991D601CA
:10018000ED91FC910190F081E02DC6010995892B3C
:1001900079F7C501DF91CF911F910F91FF90EF90FB
:1001A000DF90CF90BF90AF900895FC01538D448DA8
:1001B000252F30E0842F90E0821B930B541710F012
:1001C000CF96089501970895FC01918D828D98171F
:1001D00061F0A28DAE0FBF2FB11D5D968C91928DF7
:1001E0009F5F9F73928F90E008958FEF9FEF089528
:1001F000FC01918D828D981731F0828DE80FF11DF1
:10020000858D90E008958FEF9FEF0895FC01918D0B
:10021000228D892F90E0805C9F4F821B91098F7304
:100220009927089589EF91E00E94060121E0892B2A
:1002300009F420E0822F089580E090E0892B29F0D6
:100240000E94120181110C9400000895FC01A48DFC
:10025000A80FB92FB11DA35ABF4F2C91848D90E0E8
:1002600001968F739927848FA689B7892C93A089CB
:10027000B1898C91837080648C93938D848D981355
:1002800006C00288F389E02D80818F7D80830895E8
:10029000EF92FF920F931F93CF93DF93EC0181E0D6
:1002A000888F9B8D8C8D98131AC0E889F98980817D
:1002B00085FF15C09FB7F894EE89FF896083E889B0
:1002C000F98980818370806480839FBF81E090E0A2
:1002D000DF91CF911F910F91FF90EF900895F62E2F
:1002E0000B8D10E00F5F1F4F0F731127E02E8C8DC9
:1002F0008E110CC00FB607FCFACFE889F98980810E
:1003000085FFF5CFCE010E942601F1CFEB8DEC0FDA
:10031000FD2FF11DE35AFF4FF0829FB7F8940B8F2A
:10032000EA89FB8980818062CFCFCF93DF93EC0194
:10033000888D8823B9F0AA89BB89E889F9898C91CD
:1003400085FD03C0808186FD0DC00FB607FCF7CF89
:100350008C9185FFF2CF808185FFEDCFCE010E9489
:100360002601E9CFDF91CF91089590E0FC01E85993
:10037000FF4F2491FC01EC55FF4F3491FC01E057F5
:10038000FF4FE491EE23C9F0222339F0233001F12D
:10039000A8F4213019F1223029F1F0E0EE0FFF1F0F
:1003A000E458FF4FA591B4918FB7F894EC91611187
:1003B00026C030953E233C938FBF08952730A9F087
:1003C0002830C9F0243049F7809180008F7D03C028
:1003D000809180008F7780938000DFCF84B58F7706
:1003E00084BDDBCF84B58F7DFBCF8091B0008F774C
:1003F0008093B000D2CF8091B0008F7DF9CF3E2B9B
:10040000DACF8E50806480937C0080917A00806483
:1004100080937A0080917A0086FDFCCF80917800ED
:100420009091790008953FB7F89480917F01909161
:100430008001A0918101B091820126B5A89B05C0E1
:100440002F3F19F00196A11DB11D3FBFBA2FA92F53
:10045000982F8827BC01CD01620F711D811D911D50
:1004600042E0660F771F881F991F4A95D1F70895BC
:100470008F929F92AF92BF92CF92DF92EF92FF92B4
:100480004B015C010E9413026B017C010E9413026C
:100490006C197D098E099F09683E7340810591059D
:1004A000A8F321E0821A9108A108B10888EEC80ECD
:1004B00083E0D81EE11CF11C81149104A104B10455
:1004C00029F7FF90EF90DF90CF90BF90AF909F9073
:1004D0008F90089520915701260F3327331F213223
:1004E0003105ECF42091CF01FC0190E080E0243054
:1004F00069F082E00895A09157012191AC01495C17
:100500005E4FA40FB52FB11D2C930196861798F35B
:1005100080915701680F6093570180E0089581E052
:1005200008951092CF0181E08093CE011092A9012D
:1005300061E082E10E94B50161E083E10E94B501C2
:10054000E9EBF0E080818E7F808380818D7F8083E6
:1005500088E48093B80085E48093BC000895CF932D
:10056000DF9391E0909336018823B9F0C091B800F1
:10057000D091BA008091BC008A7B8093BC0060E07F
:1005800082E10E94B50160E083E10E94B5010E9412
:100590009102D093BA00C093B800DF91CF91089533
:1005A0000895E091880180918701E81730F4F0E028
:1005B000E757FE4F808190E008958FEF9FEF0895F9
:1005C00090918801809187012FEF3FEF981748F4B1
:1005D000E92FF0E0E757FE4F208130E09F5F9093D6
:1005E0008801C90108958091870190918801891B34
:1005F000990B0895CF92DF92EF92FF920F931F9382
:10060000CF93DF937C01CB018A012091F801222353
:1006100089F0EB016B01C40ED51ECC15DD0569F028
:100620006991D701ED91FC910190F081E02DC70116
:100630000995F3CF642F0E946A02C801DF91CF9120
:100640001F910F91FF90EF90DF90CF900895CF937F
:10065000DF931F92CDB7DEB769832091F801222383
:10066000F9F02091F501203258F021E030E0FC0152
:100670003383228390E080E00F90DF91CF91089543
:100680008091F601E82FF0E0EB52FE4F99819083C4
:100690008F5F8093F6018093F50181E090E0ECCFCD
:1006A00061E0CE0101960E946A02F7CF90E080E0FF
:1006B0000895FC0101900020E9F73197AF01481B34
:1006C000590BBC0189EF91E00C94A8008F929F9286
:1006D000AF92BF920F931F93CF93DF93CDB7DEB747
:1006E000A1970FB6F894DEBF0FBECDBF19A242305E
:1006F00008F44AE08E010F5D1F4F842E912CB12C1F
:10070000A12CA50194010E94B30CE62FB901CA01E6
:10071000EA30F4F4E05DD801EE938D01232B242B15
:10072000252B79F790E080E0109719F0CD010E9419
:100730005903A1960FB6F894DEBF0FBECDBFDF916F
:10074000CF911F910F91BF90AF909F908F90089580
:10075000E95CE1CF4F925F926F927F928F929F926E
:10076000AF92BF92CF92DF92EF92FF920F931F93BF
:10077000CF936B017C01742EAC019B010E94AE0CE7
:10078000882399F084E291E0CF911F910F91FF901F
:10079000EF90DF90CF90BF90AF909F908F907F9021
:1007A0006F905F904F900C94590346015701E89465
:1007B000B7F82FEF3FEF4FE75FE7C501B4010E94A5
:1007C000AE0C81110DC02FEF3FEF4FE75FE7C50182
:1007D000B4010E94E40A18161CF488E291E0D4CF18
:1007E0002FEF3FEF4FE75FE4C701B6010E943C0CDB
:1007F00018161CF48CE291E0C7CF2FEF3FEF4FE7C4
:100800005FECC701B6010E94E40A87FDF3CF20E048
:1008100030E0A901C701B6010E94E40A10E000E03F
:1008200087FF0AC06DE289EF91E00E9448018C01C8
:10083000F7FAF094F7F8F094C0E060E070E080E040
:100840009FE37C1641F020E030E040E251E40E945A
:10085000E90ACF5FF6CFA70196010E94780A2B0123
:100860003C010E945B0B4B015C014AE00E94660365
:100870007C01E00EF11ECC23C1F1C501B4010E9440
:100880008A0B9B01AC01C301B2010E94770A4B01A4
:100890005C016EE289EF91E00E944801E80EF91ECA
:1008A000C15018F120E030E040E251E4C501B4014C
:1008B0000E94410C2B013C010E945B0B4B01B12CAF
:1008C000A12C4AE0C501B4010E946603E80EF91E9E
:1008D000C501B4010E948A0B9B01AC01C301B201A6
:1008E0000E94770A4B015C01DBCFC701CF911F91BA
:1008F0000F91FF90EF90DF90CF90BF90AF909F90BF
:100900008F907F906F905F904F9008954F925F927D
:100910006F927F928F929F92AF92BF92CF92DF920F
:10092000EF92FF920F931F93CF93DF93A091A302B7
:10093000B091A4029091A20221E02093F80190933B
:10094000F7011092F6011092F501ED91FC911197CB
:100950000190F081E02D682FCD010995D091F5012E
:1009600081E0D13208F09CC0C091F7010E941302CF
:100970006B017C018091CF0181116CC082E080937A
:10098000CF0181E08093CE018FEF8093CD01109253
:10099000CC01D093CB01E5EDF1E0ABEAB1E080E032
:1009A000D8139AC01092AA018091AA01CC0FC82B2B
:1009B000C093AA018091A901813009F091C01092E1
:1009C000A9010E9413026B017C018091AA0180930E
:1009D000BB008091D1019091D201A091D301B0913F
:1009E000D401892B8A2B8B2BA1F00E94130200913A
:1009F000D1011091D2012091D3013091D4016C1911
:100A00007D098E099F09061717072807390708F47B
:100A100042C08091BC0083FDD8CF85EC8093BC00A0
:100A20000E9413026B017C018091CF01823009F496
:100A300059C08091CD018F3F09F476C08091CD01DE
:100A4000803209F473C08091CD01803309F470C005
:100A500084E026C08091D1019091D201A091D30170
:100A6000B091D401892B8A2B8B2B09F483CF0E9460
:100A700013020091D1011091D2012091D301309144
:100A8000D4016C197D098E099F09061717072807DD
:100A9000390708F06FCF8091D0010E94AF0285E046
:100AA0001092F6011092F5011092F801882309F4D2
:100AB00041C086EE93E0DF91CF911F910F91FF909F
:100AC000EF90DF90CF90BF90AF909F908F907F90EE
:100AD0006F905F904F90089591919D938F5F60CF3D
:100AE00085EE9CCF8091D1019091D201A091D3014C
:100AF000B091D401892B8A2B8B2B09F495CF0E94BE
:100B000013020091D1011091D2012091D3013091B3
:100B1000D4016C197D098E099F090617170728074C
:100B2000390708F081CFB7CF80E0BACF82E0B8CFE5
:100B300083E0B6CFDAE011E00FEFA2E0FA2EB5EED7
:100B4000EB2EC5ECDC2E6AE070E080E090E00E94C5
:100B50003802C091A2020E9413024B015C018091F5
:100B6000CF01811162C01093CF011093CE01009389
:100B7000CD011092CC01F092CB011093AA0180918B
:100B8000AA01CC0FC82BC093AA018091A901813082
:100B900009F0D1C01092A9010E9413024B015C011F
:100BA0008091AA018093BB008091D1019091D201E4
:100BB000A091D301B091D401892B8A2B8B2BA1F06A
:100BC0000E9413024090D1015090D2016090D30155
:100BD0007090D401681979098A099B09461657064D
:100BE0006806790608F442C08091BC0083FDD8CF26
:100BF000D092BC000E9413024B015C018091CF0196
:100C0000813009F49BC08091CC01833008F0B8C0DA
:100C10008091CC01ABEAB1E0E9E8F1E090E098170F
:100C200051F12D9121939F5FFACF8091D101909145
:100C3000D201A091D301B091D401892B8A2B8B2BA7
:100C400009F48DCF0E9413024090D1015090D2013F
:100C50006090D3017090D401681979098A099B09C1
:100C6000461657066806790608F079CF8091D001BC
:100C70000E94AF0280E01092880180938701D150DA
:100C800009F417CF833009F05ECF8091A3029091D1
:100C9000A402DC01ED91FC910284F385E02D09951D
:100CA000D82F8091A3029091A402DC01ED91FC91D8
:100CB0000284F385E02D0995C82F8091A3029091BD
:100CC000A402DC01ED91FC910284F385E02D0995ED
:100CD00020E03D2F2C2BA90170E060E0762F652FDE
:100CE000542F4427482B87E190E0C12CE0E8DE2E0A
:100CF000E8E9EE2EF12C4A015B01082E04C0B694FF
:100D0000A794979487940A94D2F780FE04C04C2548
:100D10005D256E257F25F694E794D794C7940197B7
:100D20008730910541F7C9018C7F442309F4C3CE74
:100D300087EE93E0C0CEE092BC005CCF8091D10101
:100D40009091D201A091D301B091D401892B8A2B2B
:100D50008B2B09F453CF0E9413024090D101509085
:100D6000D2016090D3017090D401681979098A0981
:100D70009B09461657066806790608F03FCF76CFDE
:100D800083E048CF85ED8093BC008091D1019091A4
:100D9000D201A091D301B091D4010796A11DB11D3C
:100DA00023E0B695A795979587952A95D1F7209139
:100DB000BC0024FD03C01092CF0108954091D101E1
:100DC0005091D2016091D3017091D401452B462BF3
:100DD000472B69F30097A105B10541F025E32A955A
:100DE000F1F700000197A109B109E1CF8091D0018D
:100DF0000C94AF021F920F920FB60F9211242F93F3
:100E00003F934F935F936F937F938F939F93AF9392
:100E1000BF93EF93FF9389EF91E00E942601FF912A
:100E2000EF91BF91AF919F918F917F916F915F9162
:100E30004F913F912F910F900FBE0F901F901895DB
:100E40001F920F920FB60F9211242F938F939F939F
:100E5000EF93FF93E0910902F0910A028081E09103
:100E60000F02F091100282FD1BC09081809112024E
:100E70008F5F8F7320911302821741F0E09112026D
:100E8000F0E0E750FE4F958F80931202FF91EF91B3
:100E90009F918F912F910F900FBE0F901F901895DB
:100EA0008081F4CF1F920F920FB60F9211242F93CF
:100EB0003F938F939F93AF93BF9380917B019091CA
:100EC0007C01A0917D01B0917E0130917A0123E0F7
:100ED000230F2D3758F50196A11DB11D20937A01DE
:100EE00080937B0190937C01A0937D01B0937E0160
:100EF00080917F0190918001A0918101B091820148
:100F00000196A11DB11D80937F0190938001A09354
:100F10008101B0938201BF91AF919F918F913F91D9
:100F20002F910F900FBE0F901F90189526E8230F5A
:100F30000296A11DB11DD2CF1F920F920FB60F9234
:100F400011242F933F934F935F936F937F938F93CE
:100F50009F93AF93BF93EF93FF938091B900887FE6
:100F6000803609F44AC0F0F5883209F4A7C018F5B4
:100F7000803109F49BC0B8F4882309F4F9C08830A3
:100F800009F494C0FF91EF91BF91AF919F918F9120
:100F90007F916F915F914F913F912F910F900FBE75
:100FA0000F901F901895883109F488C0803251F74E
:100FB0008093CD0114C0803409F49DC040F4803387
:100FC000B9F38833F9F68093CD0185ECB0C0803554
:100FD00009F485C0883509F496C0883499F60E94D2
:100FE000C206D0CF883909F48CC038F5883729F08B
:100FF00050F4883611F0803729F683E08093CF01D2
:101000001092790157C0883809F47BC0803919F0F3
:10101000803809F0B7CF80917901803208F071C033
:10102000E091790181E08E0F809379018091BB007E
:10103000F0E0E75AFE4F80833DC0803B39F0E0F49A
:10104000803A09F479C0883A09F09CCF84E0809313
:10105000CF011092580110925701E0918501F09153
:10106000860109958091570181110FC081E080931D
:1010700057011092370109C0803C09F4A6CF883C83
:1010800009F4A3CF883B09F07DCFE091580181E0BE
:101090008E0F80935801F0E0E95CFE4F80818093D1
:1010A000BB00909158018091570129C08091AA01FD
:1010B0008093BB0085EC8093BC0064CF9091CC0101
:1010C0008091CB01981758F5E091CC0181E08E0F0B
:1010D0008093CC01F0E0E555FE4F8081E9CFE091AF
:1010E000CC0181E08E0F8093CC018091BB00F0E0B9
:1010F000E555FE4F80839091CC018091CB019817EC
:10110000C8F285E8D8CFE091CC0181E08E0F8093C2
:10111000CC018091BB00F0E0E555FE4F80838091CB
:10112000CE0181115CCF81E08093A90184EA809394
:10113000BC001092CF0126CF85EC8093BC001092AA
:10114000CF0180917901803230F4E0917901F0E0B3
:10115000E75AFE4F10826091790170E0E0918301BF
:10116000F091840189E591E00995109279010ACF07
:101170001092CD0134CFE9EFF1E01382128288EEB4
:1011800093E0A0E0B0E084839583A683B78324E056
:1011900031E03183208325EC30E03587248724EC4F
:1011A00030E03787268720EC30E0318B208B21EC34
:1011B00030E0338B228B22EC30E0358B248B26EC15
:1011C00030E0378B268B118E128E138E148EE6E94B
:1011D000F2E01382128284839583A683B78386E12B
:1011E00091E091838083A2EAB2E080E48C9312962E
:1011F000FC93EE9311970895789484B5826084BD32
:1012000084B5816084BD85B5826085BD85B581600A
:1012100085BD80916E00816080936E001092810088
:101220008091810082608093810080918100816043
:101230008093810080918000816080938000809104
:10124000B10084608093B1008091B0008160809390
:10125000B00080917A00846080937A0080917A0057
:10126000826080937A0080917A00816080937A0016
:1012700080917A00806880937A001092C10084E0A7
:101280000E94870085E00E94870087E00E94870017
:1012900060E087E00E94B501E0910902F0910A0246
:1012A00082E08083E0910502F09106021082E091D5
:1012B0000702F091080280E1808310921102E09110
:1012C0000D02F0910E0286E08083E0910B02F09116
:1012D0000C02808180618083E0910B02F0910C020E
:1012E000808188608083E0910B02F0910C02808104
:1012F00080688083E0910B02F0910C0280818F7DE9
:10130000808310928801109287011092F60110924A
:10131000F5010E94910286EA90E090938601809305
:10132000850187EA90E0909384018093830164E6CD
:1013300070E080E090E00E94380200E010E089EF69
:1013400091E00E940601892B09F4BFC089EF91E06A
:101350000E94E4008337910509F081C085EF0E9467
:1013600086049C01265E3340BC0190E080E0223080
:10137000310508F056C00E948A0B6B017C0183EF97
:101380000E9486049C01265E3340BC0190E080E010
:101390002230310508F054C00E948A0B2B013C0119
:1013A00080E10E9401025C018EE00E940102EC01DA
:1013B00042E0C701B6010E94AA0380E391E00E94C7
:1013C000590342E0C301B2010E94AA0380E391E005
:1013D0000E945903B501BB0C880B990B0E948C0B22
:1013E00020E030E040EA5BE30E94410C42E00E94D2
:1013F000AA0380E391E00E945903BE01DD0F880B30
:10140000990B0E948C0B20E030E040EA5BE30E94E5
:10141000410C42E00E94AA0382E391E00E9459033A
:101420008ECF0E948A0B20E030E04AEF5AE30E9400
:10143000410C20E030E040EC50E40E94770A9DCF60
:101440000E948A0B22E538EB4FE25BE30E94410CDD
:1014500026E636E64BE352E40E94770A9FCF8836B1
:10146000910579F461E084E00E94B50164E670E0E2
:1014700080E090E00E94380260E084E00E94B501C4
:101480005ECF8936910569F461E085E00E94B5017F
:1014900064E670E080E090E00E94380260E085E061
:1014A000EDCFEC01C154D109CA31D10508F047CFC5
:1014B00061E08C2F0E94B50164E670E080E090E06E
:1014C0000E94380260E08C2FD9CF61E070E080E0AC
:1014D00090E00E9438020115110509F430CF0E94F6
:1014E0001201882309F42BCF0E94000028CF505806
:1014F000BB27AA270E948F0A0C94020C0E94F40BAF
:1015000038F00E94FB0B20F039F49F3F19F426F4C9
:101510000C94F10B0EF4E095E7FB0C94EB0BE92F28
:101520000E94130C58F3BA176207730784079507D4
:1015300020F079F4A6F50C94350C0EF4E0950B2E02
:10154000BA2FA02D0B01B90190010C01CA01A00115
:101550001124FF27591B99F0593F50F4503E68F170
:101560001A16F040A22F232F342F4427585FF3CFB1
:10157000469537952795A795F0405395C9F77EF482
:101580001F16BA0B620B730B840BBAF09150A1F0CB
:10159000FF0FBB1F661F771F881FC2F70EC0BA0F51
:1015A000621F731F841F48F4879577956795B795D9
:1015B000F7959E3F08F0B0CF9395880F08F09927D4
:1015C000EE0F9795879508950E94C70B08F481E068
:1015D00008950E94FD0A0C94020C0E94FB0B58F027
:1015E0000E94F40B40F029F45F3F29F00C94EB0BC0
:1015F00051110C94360C0C94F10B0E94130C68F3EF
:101600009923B1F3552391F3951B550BBB27AA27BB
:1016100062177307840738F09F5F5F4F220F331FF5
:10162000441FAA1FA9F335D00E2E3AF0E0E832D0BD
:1016300091505040E695001CCAF72BD0FE2F29D0C0
:10164000660F771F881FBB1F261737074807AB0792
:10165000B0E809F0BB0B802DBF01FF2793585F4F07
:101660003AF09E3F510578F00C94EB0B0C94360C3D
:101670005F3FE4F3983ED4F3869577956795B795E9
:10168000F7959F5FC9F7880F911D9695879597F9F4
:101690000895E1E0660F771F881FBB1F621773076D
:1016A0008407BA0720F0621B730B840BBA0BEE1F82
:1016B00088F7E09508950E941B0C88F09F5798F0DA
:1016C000B92F9927B751B0F0E1F0660F771F881F47
:1016D000991F1AF0BA95C9F714C0B13091F00E9461
:1016E000350CB1E008950C94350C672F782F8827BE
:1016F000B85F39F0B93FCCF3869577956795B39588
:10170000D9F73EF490958095709561957F4F8F4FF6
:101710009F4F0895E89409C097FB3EF490958095FB
:10172000709561957F4F8F4F9F4F9923A9F0F92FA7
:1017300096E9BB279395F695879577956795B79525
:10174000F111F8CFFAF4BB0F11F460FF1BC06F5F0B
:101750007F4F8F4F9F4F16C0882311F096E911C01D
:10176000772321F09EE8872F762F05C0662371F03E
:1017700096E8862F70E060E02AF09A95660F771F52
:10178000881FDAF7880F9695879597F90895990F2E
:101790000008550FAA0BE0E8FEEF16161706E8073B
:1017A000F907C0F012161306E407F50798F0621B5C
:1017B000730B840B950B39F40A2661F0232B242B31
:1017C000252B21F408950A2609F4A140A6958FEF50
:1017D000811D811D089597F99F6780E870E060E0A2
:1017E00008959FEF80EC089500240A9416161706BA
:1017F00018060906089500240A9412161306140602
:1018000005060895092E0394000C11F4882352F064
:10181000BB0F40F4BF2B11F460FF04C06F5F7F4F1C
:101820008F4F9F4F089557FD9058440F551F59F003
:101830005F3F71F04795880F97FB991F61F09F3FBD
:1018400079F087950895121613061406551FF2CFE6
:101850004695F1DF08C0161617061806991FF1CF36
:1018600086957105610508940895E894BB2766275D
:101870007727CB0197F908950E94C70B08F48FEFE3
:1018800008950E94540C0C94020C0E94F40B38F042
:101890000E94FB0B20F0952311F00C94EB0B0C94A1
:1018A000F10B11240C94360C0E94130C70F3959FCD
:1018B000C1F3950F50E0551F629FF001729FBB2747
:1018C000F00DB11D639FAA27F00DB11DAA1F649FE3
:1018D0006627B00DA11D661F829F2227B00DA11D96
:1018E000621F739FB00DA11D621F839FA00D611D1C
:1018F000221F749F3327A00D611D231F849F600D3D
:10190000211D822F762F6A2F11249F5750409AF065
:10191000F1F088234AF0EE0FFF1FBB1F661F771FF1
:10192000881F91505040A9F79E3F510580F00C94BC
:10193000EB0B0C94360C5F3FE4F3983ED4F38695A2
:1019400077956795B795F795E7959F5FC1F7FE2B5C
:10195000880F911D9695879597F908950E94C70B5A
:10196000880B990B0895A1E21A2EAA1BBB1BFD013F
:101970000DC0AA1FBB1FEE1FFF1FA217B307E4076E
:10198000F50720F0A21BB30BE40BF50B661F771FC6
:10199000881F991F1A9469F76095709580959095A6
:1019A0009B01AC01BD01CF010895EE0FFF1F059013
:1019B000F491E02D0994F894FFCF00000000480155
:1019C000A800D50095010601E400F8000000000021
:1019D0002703FA025603D002F302E002D1026E613D
:1019E0006E00696E66006F7666002C000D0A0000BE
:107E0000112484B714BE81FFF0D085E080938100F7
:107E100082E08093C00088E18093C10086E0809377
:107E2000C20080E18093C4008EE0C9D0259A86E02C
:107E300020E33CEF91E0309385002093840096BBD3
:107E4000B09BFECF1D9AA8958150A9F7CC24DD24C4
:107E500088248394B5E0AB2EA1E19A2EF3E0BF2EE7
:107E6000A2D0813461F49FD0082FAFD0023811F036
:107E7000013811F484E001C083E08DD089C08234E0
:107E800011F484E103C0853419F485E0A6D080C0E4
:107E9000853579F488D0E82EFF2485D0082F10E0AE
:107EA000102F00270E291F29000F111F8ED06801E7
:107EB0006FC0863521F484E090D080E0DECF843638
:107EC00009F040C070D06FD0082F6DD080E0C81688
:107ED00080E7D80618F4F601B7BEE895C0E0D1E017
:107EE00062D089930C17E1F7F0E0CF16F0E7DF06D8
:107EF00018F0F601B7BEE89568D007B600FCFDCFD4
:107F0000A601A0E0B1E02C9130E011968C91119780
:107F100090E0982F8827822B932B1296FA010C0160
:107F200087BEE89511244E5F5F4FF1E0A038BF0790
:107F300051F7F601A7BEE89507B600FCFDCF97BE46
:107F4000E89526C08437B1F42ED02DD0F82E2BD052
:107F50003CD0F601EF2C8F010F5F1F4F84911BD097
:107F6000EA94F801C1F70894C11CD11CFA94CF0C13
:107F7000D11C0EC0853739F428D08EE10CD085E9AC
:107F80000AD08FE07ACF813511F488E018D01DD067
:107F900080E101D065CF982F8091C00085FFFCCF94
:107FA0009093C60008958091C00087FFFCCF809118
:107FB000C00084FD01C0A8958091C6000895E0E648
:107FC000F0E098E1908380830895EDDF803219F02E
:107FD00088E0F5DFFFCF84E1DECF1F93182FE3DFCA
:107FE0001150E9F7F2DF1F91089580E0E8DFEE27F6
:047FF000FF270994CA
:027FFE00040479
:00000001FF
